:030000000247AF05
:0C47AF0078FFE4F6D8FD7581630247F640
:101EC1000A53746172743A20004950436F6E6E6513
:101ED10063745245510A004950436F6E6E656374D5
:101EE100003E432C562C43432CC0E4E0EFF2E5F0D6
:101EF10020D1E8EDEAEEEC49500A003E432C4D4179
:101F0100432C25303262583A25303262583A253016
:101F11003262583A25303262583A25303262583AA4
:101F210025303262582C4D414320E0E4F0E5F10ABE
:101F3100003E432C5645522C20332E3020EEF22009
:101F410025732025732CC2E5F0F1E8FF20495020CC
:101F5100ECEEE4F3EBFF0A004F63742030332032E0
:101F61003030370031323A30313A3239003E432C89
:101F71004C442C50524F473A202020202020202032
:101F81002020202020202020202020202020202050
:101F91002020202020202020202020202020202040
:101FA1002020202020202020202020202020202030
:101FB100202020202020202020202020202CC4E0B0
:101FC100F2E020EFF0EEF8E8E2EAE828F4E0E9EBED
:101FD100290A003E2A2C312CCEF1EDEEE2EDFBE593
:101FE10020EFE0F0E0ECE5F2F0FB20F1E5F2E5E2D4
:101FF100EEE3EE20E8EDF2E5F0F4E5E9F1E00A00C8
:102001003E412C4130312C2562752E2562752E25DD
:1020110062752E2562752C495020E0E4F0E5F1202F
:10202100E0E4E0EFF2E5F0E00A003E412C4130321D
:102031002C2562752E2562752E2562752E256275F9
:102041002C495020E0E4F0E5F120EEF1ED2E20F1F5
:10205100E5F0E2E5F0E00A003E412C4130332C2569
:1020610062752E2562752E2562752E2562752C49A5
:102071005020E0E4F0E5F120F0E5E72E20F1E5F075
:10208100E2E5F0E00A003E412C4130342C25627536
:102091002E2562752E2562752E2562752CCCE0F1F8
:1020A100EAE020F1E5F2E80A003E412C4130352C0E
:1020B1002562752E2562752E2562752E2562752C79
:1020C100D8EBFEE70A003E532C4130362C256275D1
:1020D1002CC2F0E5ECFF20EEE6E8E42E20EAE2E88F
:1020E100F2E0EDF6E8E820282A3130ECF1290A0087
:1020F1003E2A2C312CC4EEEF2E20EFE0F0E0ECE58F
:10210100F2F0FB20F1E5F2E5E2EEE3EE20E8EDF29C
:10211100E5F0F4E5E9F1E00A003E422C5330312CC0
:102121002562752CC6E4E0F2FC20E7E0EFF0EEF169
:10213100E020F1EEE5E4E8EDE5EDE8FF20EEF22048
:10214100F1E5F0E2E5F0E00A003E422C5330322C9A
:102151002562752C43E2FFE7FC20F120F1E5F0E276
:10216100E5F0EEEC20EDE520EFEEE4E4E5F0E6E865
:10217100E2E0F2FC0A003E422C5330332C2562751A
:102181002CCFE5F0E5E7E0EFF3F1EA20EFF0E8200E
:10219100EFEEF2E5F0E520F1E2FFE7E820F120F1D2
:1021A100E5F0E2E5F0EEEC0A003E422C5330342C2F
:1021B1002562752CCDE5F220EFE5F0E5E4E0F7E8E6
:1021C10020E4E8E0E3EDEEF1F2E8EAE820E220F1D4
:1021D100E5F0E2E5F00A003E422C5330352C256251
:1021E100752CCAE0EDE0EB20F8E8F0EEEAEEE2E56E
:1021F100F8E0F2E5EBFCEDEEE3EE20EEE1ECE5EDEF
:10220100E00A003E532C5330362C253032625825DB
:1022110030326258253032625825303262582530CA
:1022210032625825303262582C4D414320E0E4F0AF
:10223100E5F120F8E8F0EEEAEEE2E5F8E0F2E5EBB0
:10224100FCEDEEE3EE20EEE1ECE5EDE00A003E45CB
:102251004E440A0044756D705820202020203030F3
:1022610020303120303220303320303420303520BE
:10227100303620303720303820303920304120307E
:10228100422030432030442030452030460A003A75
:1022910020000A0044756D70442020202020303039
:1022A100203031203032203033203034203035207E
:1022B100303620303720303820303920304120303E
:1022C100422030432030442030452030460A00452A
:1022D1007272206B657900526420656570726F6D52
:1022E1000A005264204D454D0A00526420436F6438
:1022F100650A0044656275674950204F4E0A0044E3
:10230100656275674950204F46460A00446562750B
:102311006755736572204F6E0A0044656275675593
:10232100736572204F46460A0044656275674D73B6
:1023310067204F6E0A0044656275674D7367204FD1
:1023410046460A00436F6E666967206C6F636B21B6
:102351000A00577220656570726F6D0A0020536123
:10236100766520656570726F6D210A004572722075
:102371004D414321004C6F61643E3E002A003C41C7
:1023810030313D003C4130323D003C4130333D0075
:102391003C4130343D003C4130353D003C4130361C
:1023A1003D004E4F4950004C494E4B434F4E545205
:1023B100005452415353004652004E4F4C494E4B2C
:1023C10000494E49004E4F4449414700003C21001D
:1023D1003C5330313D003C5330323D003C533033AF
:1023E1003D003C5330343D003C5330353D003C53BF
:1023F10030363D00FF23A3FF23A8FF23B2FF23B8FC
:0C240100FF23BBFF23C2FF23C6FF23CD37
:06520F00016000015E00D9
:1051A300C2AFC28E758900438910758BFF758DB7A9
:0751B300D2ABD28ED2AF2275
:03001B0002471980
:10471900C0E0C083C082C0D0C2AFC28E758BFF75A6
:104729008DB720190675A61E75A6E1055ED215E599
:104739006060020560E55FD394014002155F05637F
:10474900E563540F704AD220E563543F7014D213C5
:10475900906ECCE0600C04F0E0D394B44004C2AF96
:1047690080FE906EC7E0600204F0906943E0600249
:1047790014F0906ECDE0D394014003E014F03018AA
:10478900020561E562D394644004D219800205628E
:10479900E55DD394014002155DD28ED2AFD0D0D061
:0647A90082D083D0E03253
:1018A900C291C290D2B5C21D7D027C007F07125140
:1018B900378F27E527646060097D017F601250CB6F
:1018C900D21DE4FDFC7F0B1251378F27E52730E647
:1018D900097D04E4FF1250EFD21D7D017C007F07D2
:1018E9001251378F27E5277008FD7FFF1250CBD2A1
:1018F9001D301D03126000C2AFC288C2A8C2AA125D
:101909004A44906B80E0B4FA09A3E064CE70030204
:1019190019A0E4F52774782527F582E4346BF5835B
:10192900E4F00527E527B443EC906B8074FAF0A343
:1019390074CEF0A374CCF0906B86740AF0E4A3F033
:10194900A304F0A3F0906B8B7403F0A374CCF09014
:101959006B7C74FFF0A3F0A3F0E4A3F0906B977491
:1019690005F0E4F527E5272401FFE433FE74782523
:1019790027F582E4346BF583E0FD12518A0527E5EA
:1019890027C3944340DFE4F5A775A61E75A6E19029
:101999007FF0F0A3F080FED2AF906B8B7403F0A3BD
:1019A90074CCF0E4906B8AF012417DEF600312323F
:1019B9008FC2B5123482C219124E81906B97E0C35F
:1019C900940350037403F0D21FD21ED21DD2932068
:1019D9001D077E1E7FC1124263E4906DB7F012515C
:1019E900A3C2AFA37408F0906AF67424F0E4A3F0DC
:1019F900906B80E0906AF8F0906B81E0906AF9F062
:101A0900906B82E0906AFAF0906B83E0906AFBF049
:101A1900906B84E0906AFCF0906B85E0906AFDF031
:101A2900755F01E4906DB9F0C21AC21BD2AF75A7F8
:101A39000775A61E75A6E11250A5201D19AF277EB0
:101A4900007D03124344E4FF12466F7E6B7FB7E4C7
:101A5900FB7D0112441E906ECCE060037401F0E43A
:101A6900906943F0A37455F0A37481F0E4F561E43F
:101A7900F562906943E07003122769906ECDE0B476
:101A890001119080007410F0E4906ECDF0D21DD257
:101A99001ED21F908008E0F52730E405D21A741091
:101AA900F0E52730E508D21C9080087420F0E5277E
:101AB90030E608D21B9080087440F0E561D39403A6
:101AC9004023908002E4F0908001F0908000F0E5DE
:101AD90061D39406400FE4F561C216906DB9F075B3
:101AE9005F01124E819080A0E07003124B3D9080FF
:101AF900B8E07003124BB79080D0E07003124CFF2E
:101B0900908000E07013301A10124079906B73EFD7
:101B1900F0D394004003120A1A908002E0700690F4
:101B29008000E06005D218021A78C218E4F56190C5
:101B39006943E06003021A78301C12123CC9906BA9
:101B490073EFF0D394004005E0FF1251E2201B032C
:101B5900021CD7123B54906B73EFF07003021A7892
:101B6900906BB7E054BF247F7003021C3A147003D2
:101B7900021C1224026003021C6D201D077E1E7FB9
:101B8900CA124263302179201676906B8FE0700675
:101B9900906B93E0605B906EC3E0FF906B8FE0B554
:101BA9000724906EC4E0FE906B90E0B50618906E25
:101BB900C5E0FE906B91E0B5060C906EC6E0FE9014
:101BC9006B92E06E602B906B93E06F7033906EC4F4
:101BD900E0FF906B94E0B50727906EC5E0FF906B2E
:101BE90095E0B5071B906EC6E0FF906B96E0B507D0
:101BF9000F906DB97401F0120021755F01021CD7B5
:101C0900906EC374FFF0021CD7906ECCE060037431
:101C190001F0906EBBE0FF906BB9E06F6003021CAE
:101C2900D7906EBBE004F0E4F55F906DB7F0021C4D
:101C3900D7301603021CD7906B86E07003021A781E
:101C4900125216D216E4F55F906DB7F0906EC70484
:101C5900F0E4906EBAF0A3F0201D737E1E7FD812B7
:101C69004263806A906ECCE060037401F0301652D2
:101C7900906BB7E020E74B906BB9E0FF906EBAE04C
:101C8900FE6F600D906EC2E07007EE146F703F80BA
:101C990013906EBAE004F0906B73E0FFD3940440A4
:101CA90003124F6490683F7482F0A37401F0906B43
:101CB900B9E0906841F07E687F3F7D03124AC20215
:101CC9001A78302109201606906EC374FFF0201689
:101CD90003021D8CE55F706B124FA2EF60207E6CD2
:101CE9007FB7906CB8E02404FD124AC2906EC2E03E
:101CF9006003021A78906B97E0F55F021A78906E8C
:101D0900C7E0D3943C403C906EC2E07036906EC7F9
:101D190004F0906AF5E0702B1251FCE4906CB7F076
:101D2900A37412F0906EBBE0906CB9F0A374FDF04F
:101D390090694663A201906CBB63A2017F121237BE
:101D490046809B1251F1EF601590683F7483F0E46F
:101D5900A3F07E687F3F7D02124AC2021A78E55FCE
:101D690064016003021A78906DB7E004F0E0C3944F
:101D7900055003021CE7C216E4906DB9F012002168
:101D8900021A78E55F64016003021A78906DB9E080
:101D990014604024FE603C147003021E7424046025
:101DA90003021A78E4F561202113906DB97404F0E7
:101DB900906DB7E05401F0755F01021A78E4906DF7
:101DC900B9F0906DB704F0755FC8906EC374FFF0F9
:101DD900021A78906EC3E07003021E63906CB774A8
:101DE90080F0906CB97401F0E4A3F0A304F0A3743B
:101DF90030F0A3747BF0E4F52774BE2527F582E45F
:101E0900346CF583747DF074BF2527F582E4346C56
:101E1900F583E4F0E5272407906CB8F07C6E7DC368
:101E2900906B8BE0FAA3E0FB7F021248C07E6C7FC7
:101E3900B7E5272409FD124AC2906EC2E0601B1261
:101E49005216D216E4F55F906DB7F0906EC704F0A4
:101E5900E4906EBAF0A3F0021A78906DB97404F0A8
:101E6900906B97E02432F55F021A78908002741023
:101E7900F0755F03906DB7E06401FFF0906DB97480
:101E890001F0EF7019906B93E06013FCA3E0FDA3E0
:101E9900E0FEA3E0FF906EC3122C0D021A78906B3E
:101EA9008FE0FCA3E0FDA3E0FEA3E0FF906EC31268
:071EB9002C0D021A7880FED7
:011EC00022FF
:100A1A00906BB8E0B444047F0180027F00906BB70A
:100A2A00E0B447047E0180027E00EE5F604A906B6C
:100A3A0080E0906BB9F0906B81E0906BBAF0906BAC
:100A4A0082E0906BBBF0906B83E0906BBCF0906B94
:100A5A0084E0906BBDF0906B85E0906BBEF0906B7C
:100A6A00B87452F0906AEF63A2019080A863A20161
:100A7A007F06123746021253906B73E0C3940850F4
:100A8A000302125C906B80E0FF906BB9E06F600329
:100A9A0002125C906B81E0FF906BBAE06F60030218
:100AAA00125C906B82E0FF906BBBE06F60030212F6
:100ABA005C906B83E0FF906BBCE06F600302125C9A
:100ACA00906B84E0FF906BBDE06F600302125C9054
:100ADA006B85E0FF906BBEE06F600302125C906B67
:100AEA00B8E0B44415906AEFE0B4FF0E63A2019037
:100AFA0080A863A2017F06123746906ECCE060039D
:100B0A007401F0906ECD7464F0906BB87452F090EA
:100B1A006BB7E0646D6003020C977BFF7A1E79E283
:100B2A0012246F7BFF7A1E79FC906B80E0F530A36C
:100B3A00E0F531A3E0F532A3E0F533A3E0F534A301
:100B4A00E0F53512246F7530FF75311F753259750E
:100B5A0033FF75341F7535657BFF7A1F793212248E
:100B6A006F7BFF7A1F796E12246F7BFF7A1F79D40D
:100B7A0012246F7BFF7A207901906B86E0F530A30F
:100B8A00E0F531A3E0F532A3E0F53312246F7BFFE1
:100B9A007A20792B906B8FE0F530A3E0F531A3E052
:100BAA00F532A3E0F53312246F7BFF7A207959904E
:100BBA006B93E0F530A3E0F531A3E0F532A3E0F55D
:100BCA003312246F7BFF7A207987906B7CE0F530B3
:100BDA00A3E0F531A3E0F532A3E0F53312246F7BED
:100BEA00FF7A2079AA906B78E0F530A3E0F531A37B
:100BFA00E0F532A3E0F53312246F7BFF7A2079C740
:100C0A00906B97E0F53012246F7BFF7A2079F1120E
:100C1A00246F7BFF7A21791AA221E433F53012245A
:100C2A006F7BFF7A21794A906EC2E0F53012246F09
:100C3A007BFF7A217977906ECCE0F53012246F7BB6
:100C4A00FF7A2179AA906AF5E0F53012246F7BFFCA
:100C5A007A2179D8A214E433F53012246F7BFF7A13
:100C6A00227904906EBCE0F530A3E0F531A3E0F5FB
:100C7A0032A3E0F533A3E0F534A3E0F53512246F8F
:100C8A00123F637BFF7A22794F12246F22906BB74F
:100C9A00E0644C70527E227F55124263906BBFE033
:100CAA00F528A3E0F529E4F52A7D03AF29AE281239
:100CBA0043447E227F90124263AE28AF29E4FB7D33
:100CCA001012441E7E227F9312426374102529F566
:100CDA0029E43528F528052AE52AC3941040CA7E56
:100CEA00227F9312426322906BB7E0646C705CF5CA
:100CFA002C7E227F95124263E4F52BAF2C7E007D79
:100D0A00031243447E227F90124263E4F52AA82C00
:100D1A00E6FF74C1252AF582E4346BF583EFF0050A
:100D2A002C052AE52AB410E67E6B7FC1E4FB7D1010
:100D3A0012441E7E227F93124263052BE52BC39435
:100D4A000840B87E227F9312426322906BB7E06418
:100D5A004B7061F52A74A9252AF582E4346BF58370
:100D6A00E0603274A9252AF582E4346BF583E0F455
:100D7A00602374A9252AF582E4346BF583E0FF74B5
:100D8A00BF252AF582E4346BF583E0B50710052AFE
:100D9A00E52AB408C09069437432F0021253906B8A
:100DAA00B77421F0301D030212537E227FD0124203
:100DBA0063021253906BB7E0B4521A201D077E22C9
:100DCA007FD8124263906BB77472F07E6B7FB77DE7
:100DDA000812494422906BB7E064497045201D0708
:100DEA007E227FE3124263906BBFE0F528A3E0F511
:100DFA0029E4F52A852982852883E0FF74C1252AFA
:100E0A00F582E4346BF583EFF00529E529700205D4
:100E1A0028052AE52AB480DC7E6B7FB77D8A1249D1
:100E2A004422906BB7E064437079A3E06452704641
:100E3A00201D077E227FEB124263906BBFE0F528EC
:100E4A00A3E0F529E4F52A852982852883E493FF1E
:100E5A0074C1252AF582E4346BF583EFF00529E5A0
:100E6A002970020528052AE52AB480DB7E6B7FB744
:100E7A007D8A12494422906BB8E0645760030212DB
:100E8A005C906BBFE0F528A3E0F52974C1252AF52B
:100E9A0082E4346BAD82FC7B80AF29AE28125018F5
:100EAA00021253906BB7E064446003020F3E906BEA
:100EBA00BFE0FF64447003021253EFB4310CC21D49
:100ECA007E227FF4124263021253906BBFE0B43069
:100EDA000CD21D7E237F00124263021253906BBF15
:100EEA00E0B4320CD21E7E237F0D124263021253EB
:100EFA00906BBFE0B4330CC21E7E237F1B12426389
:100F0A00021253906BBFE0B4340CD21F7E237F2AA7
:100F1A00124263021253906BBFE0B4350CC21F7EBB
:100F2A00237F37124263021253906BBFE0FF120015
:100F3A001E021253906943E07013201D077E237F1F
:100F4A0045124263906BB77421F0021253906943C1
:100F5A007432F0906BB7E0FFB45104C2AF80FEEF79
:100F6A0064577045201D077E237F53124263906B9E
:100F7A00C0E0906B73F0E4F52A906B73E0FFE52A0A
:100F8A00C39F400302125374C1252AF582E4346BCD
:100F9A00F583E0FF906BBFE0252A24EEF582E43466
:100FAA0069F583EFF0052A80D0906BB7E06453604F
:100FBA0003021061201D077E237F5E124263906B3D
:100FCA0080E0FF9069F7E06F703C906B81E0FF90E2
:100FDA0069F8E06F7030906B82E0FF9069F9E0B5D4
:100FEA000724906B83E0FF9069FAE0B50718906BCD
:100FFA0084E0FF9069FBE0B5070C906B85E0FF90F9
:10100A0069FCE06F6016906BB77421F0301D030223
:10101A0012537E237F6D124263021253E4F52AE4CF
:10102A00F562AF2AFE74EE252AF582E43469F58367
:10103A00E0FD12518A052AE52AC394FE40E1C2AFB7
:10104A00E4907FF0F0A3F0907FFD74AAF0A374FF00
:10105A00F0A37455F080FE906BB7E0644F704C902B
:10106A006BBFE0F528A3E0F529E5294528700A2099
:10107A001D077E237F76124263201D077E237F7D14
:10108A00124263E4F52A74C1252AF582E4346BF529
:10109A0083E0852982852883F00529E529700205E0
:1010AA0028052AE52AB480DE021253906BB7E0FFC6
:1010BA00B44521906BBFE0FDA3E0907FF0CDF0A393
:1010CA00EDF0C2AF907FFD74AAF0A374FFF0A37491
:1010DA0055F080FEEF64656003021253906BBFE027
:1010EA00FFA3E0907FF0CFF0A3EFF0E4F528F52915
:1010FA00D3907FF1E09529907FF0E095284020E495
:10110A00F5622529FFE5283401FE85298285288391
:10111A00E0FD12518A0529E5297002052880D17E51
:10112A00237F7F12483BEF4E6020120003906B86AC
:10113A00EFF0120003906B87EFF0120003906B88B8
:10114A00EFF0120003906B89EFF07E237F8512483F
:10115A003BEF4E6020120003906B8FEFF0120003FA
:10116A00906B90EFF0120003906B91EFF012000376
:10117A00906B92EFF07E237F8B12483BEF4E6020FC
:10118A00120003906B93EFF0120003906B94EFF050
:10119A00120003906B95EFF0120003906B96EFF03C
:1011AA007E237F9112483BEF4E6020120003906B22
:1011BA007CEFF0120003906B7DEFF0120003906B4E
:1011CA007EEFF0120003906B7FEFF07E237F971281
:1011DA00483BEF4E6020120003906B78EFF012004C
:1011EA0003906B79EFF0120003906B7AEFF0120024
:1011FA0003906B7BEFF07E237F9D12483BEF4E609E
:10120A0008124E24906B97EFF0E4F52AE4F562E5B4
:10121A002A2401FFE433FE7478252AF582E4346B2C
:10122A00F583E0FD12518A052AE52AC3944340DC7E
:10123A00C2AFE4907FF0F0A3F0907FFD74AAF0A310
:10124A0074FFF0A37455F080FE7E6B7FB77D0812A1
:02125A00494405
:01125C00226F
:104FE000AE07EEC39430400BEED394395005EE2457
:104FF000D0FF22EEC39461400BEED394665005EED1
:1050000024A9FF22EEC39441400BEED394465005F1
:08501000EE24C9FF22AF0622C5
:10517000906AEEE004F07006906AEDE004F0906A48
:0A518000EDE0FEA3E0FF12515422FF
:10000300125170124FE0EFC454F0FEC0061251704B
:08001300124FE0D0E02FFF22A4
:104E2400E4906FF8F0125170906FF9EFF0C3943082
:104E34004018E0FFD394395011906FF8E02446F500
:104E440082E43469F583EFF08011906FF8E0244632
:104E5400F582E43469F583E4F0800C906FF8E004A3
:104E6400F0E0D3940840BE75330075340075350006
:0C4E7400E4F5367B017A69794612381D9E
:014E8000220F
:04483B008E2D8F2E01
:10483F00906AEDE4F0A374FFF0125170EF606EF424
:10484F00606B852E82852D83E493B507EC752F0160
:10485F00E52E252FF582E4352DF583E49360259021
:10486F006AEEE0252FFF906AEDE03400FE125154FE
:10487F00E52E252FF582E4352DF583E493B5070456
:10488F00052F80CCE52E252FF582E4352DF583E419
:10489F009370A6E52F24FFFFE434FFFE906AEEE04D
:1048AF002FF0906AEDE03EF07E007F0122E4FEFFE4
:0148BF0022D6
:10417D007E237FCE12483BEF4E70037F01227E23BC
:10418D007FD112483BEF4E600C125170EF24D024BA
:10419D00FF92218002D2217E237FD712483BEF4E22
:1041AD00600C125170EF24D0906EC2F08005E49037
:1041BD006EC2F07E237FDD12483BEF4E600C125134
:1041CD0070EF24D0906ECCF08005E4906ECCF07E34
:1041DD00237FE312483BEF4E600C125170EF24D059
:1041ED00906AF5F08005E4906AF5F07E237FE91280
:1041FD00483BEF4E600C125170EF24D024FF921407
:10420D008002C214906B8063A201906EBC63A20108
:10421D007F0612374630143B7E237FEF12483BEF6B
:10422D004E6030120003906EBCEFF0120003906EE2
:10423D00BDEFF0120003906EBEEFF0120003906E12
:10424D00BFEFF0120003906EC0EFF0120003906EFE
:06425D00C1EFF07F00221A
:10328F00C214E4906ECCF0D221C217906EC2F090AF
:10329F006AF5F0906B8063A201906EBC63A2017F10
:1032AF0006123746E4F528E52875F003A424F5F552
:1032BF0082E43423F583E493FB740193FA7402934D
:1032CF00F9122A857003023481E4F529F52AFD7479
:1032DF006E2DF582E43469F583E0FF700302347CD0
:1032EF00E52875F003A424F5F582E43423F583E48F
:1032FF0093FB740193FA740293F985298275830005
:10330F00122A9EFEEFB50608752A010529023478A8
:10331F00E52A7003023478EE6003023473E5282443
:10332F00FE602814700302345B14700302345F14C0
:10333F00700302346714700302346B2405600302B8
:10334F00347C906ECC7401F002347CD214746E2DE8
:10335F00F582E43469F583E0FF642D700302347C59
:10336F00124FE0EFC454F0FC746F2DF582E4346912
:10337F00F583E0FF124FE0EF2C906EBCF074702DD0
:10338F00F582E43469F583E0FF124FE0EFC454F0A7
:10339F00FC74712DF582E43469F583E0FF124FE080
:1033AF00EF2C906EBDF074722DF582E43469F583C5
:1033BF00E0FF124FE0EFC454F0FC74732DF582E47C
:1033CF003469F583E0FF124FE0EF2C906EBEF0747E
:1033DF00742DF582E43469F583E0FF124FE0EFC4FA
:1033EF0054F0FC74752DF582E43469F583E0FF1217
:1033FF004FE0EF2C906EBFF074762DF582E43469B8
:10340F00F583E0FF124FE0EFC454F0FC74772DF515
:10341F0082E43469F583E0FF124FE0EF2C906EC029
:10342F00F074782DF582E43469F583E0FF124FE0F4
:10343F00EFC454F0FC74792DF582E43469F583E020
:10344F00FF124FE0EF2C906EC1F08021D217801D3C
:10345F00906EC27401F08015C2218011906AF574CC
:10346F0001F08009E4F52AF5290D0232DE05280264
:02347F0032B663
:013481002228
:104EDA00906DB8E0C3947C503D906DB8E0FE04F04C
:104EEA0074F62EF582E4346AF583EFF0BF0A279050
:104EFA006DB8E0FF04F074F62FF582E4346AF583A6
:104F0A00E4F0906DB8E0FF1249C6906DB87408F0ED
:074F1A00906AF7E004F022A9
:104E81009080007480F0906B7863A201F583F582C5
:104E910063A2017F08123746906B8063A201908064
:104EA1008863A2017F0A123746908092E4F0A374CE
:104EB10032F0A37401F0906B8AE0FF9080B1F09022
:104EC10080E1EFF09080957455F0A3F0908000742C
:094ED10001F09080097470F022D8
:104B3D00908009E04410F09080A0E0706C9080A10E
:104B4D007482F09080A874FFF0A3F0A3F0A3F07F1F
:104B5D00039080AEEFF07FCBA3EFF07F039080AC9E
:104B6D00EFF0A374CBF09080007402F0906FEC1214
:104B7D002C1900000000906FECE0908040F0906FD9
:104B8D00EDE0908041F0906FEEE0908042F0906FFC
:104B9D00EFE0908043F0A3E4F0A3F0A3F0A3F09036
:094BAD008018F0A3F0A3F0A3F0BE
:014BB60022DC
:104CFF00908009E04440F09080D17482F0906B8BEB
:104D0F00E0FF9080DEF0906B8CE0FF9080DFF09002
:104D1F0080027402F0906FF0122C190000000090C6
:104D2F006FF0E0908058F0906FF1E0908059F09024
:104D3F006FF2E090805AF0906FF3E090805BF0A3F9
:104D4F00E4F0A3F0A3F0A3F0908030F0A3F0A3F071
:024D5F00A3F0BF
:014D6100222F
:104BB700908009E04420F09080B8E0706C9080B954
:104BC7007482F07F039080C6EFF07FCDA3EFF07F74
:104BD700039080C4EFF0A374CDF09080C074FFF011
:104BE700A3F0A3F0A3F09080017402F0906FF41289
:104BF7002C1900000000906FF0E090804CF0906F4F
:104C0700F1E090804DF0906FF2E090804EF0906F61
:104C1700F3E090804FF0A3E4F0A3F0A3F0A3F090AB
:094C27008024F0A3F0A3F0A3F037
:014C30002261
:1048C0008C288D29A907EAFDE975F018A424ACFF0E
:1048D000E5F034808F82F583EDF0EBFDE975F0189B
:1048E000A4FFAEF024ACFBEE34808B82F583A3ED05
:1048F000F08529828C83E0FDEF24A8FFEE3480FE52
:104900008F82F583EDF08529828C83A3E08F828EE0
:1049100083A3F0852982852883A3A3E0FDE975F0B0
:1049200018A424A8FFE5F03480FE8F82F583A3A3AA
:10493000EDF08529828C83A3A3A3E08F828E83A3CD
:04494000A3A3F0221B
:064944008D2DAB07AA0651
:10494A00906FECE0FCA3E0FDA3E0FEA3E0F5318E5E
:10495A00308D2F8C2EAE02AF038E838F8263A2011D
:10496A00E530540744C0F58385318263A201AF2D37
:10497A001237AF908000E020E5F9E4FCFDFEE53156
:10498A00252DF531EE3530F530ED352FF52FEC3597
:10499A002EF52E908040E52EF0A3E52FF0A3E5300A
:1049AA00F0A3E531F09080007420F0AF31AE30AD65
:0B49BA002FAC2E906FEC122C0DAF2DD7
:0149C50022CF
:064AC2008D28AB07AA06D7
:104AC800906FF0E0FCA3E0FDA3E0FEA3E0F52C8EE0
:104AD8002B8D2A8C29AE02AF038E838F8263A201AD
:104AE800E52B540744D0F583852C8263A201AF28B7
:104AF8001237AFE4FCFDFEE52C2528F52CEE352B0E
:104B0800F52BED352AF52AEC3529F529908058E55D
:104B180029F0A3E52AF0A3E52BF0A3E52CF090807B
:104B2800027420F0AF2CAE2BAD2AAC29906FF01296
:044B38002C0DAF2869
:014B3C002256
:02466F008F2991
:10467100908001E030E5037F0022906FF4E0FCA31D
:10468100E0FDA3E0FEA3E0F52D8E2C8D2B8C2A906E
:104691006EBC63A201E52C540744C8F583852D82C5
:1046A10063A2017F061237C5E52D2406F52DE435F9
:1046B1002CF52CE4352BF52BE4352AF52A906DBA2F
:1046C10063A201E52C540744C8F583852D8263A2BA
:1046D10001AF291237C5E4FCFDFEE52D2529F52D95
:1046E100EE352CF52CED352BF52BEC352AF52A90F2
:1046F100804CE52AF0A3E52BF0A3E52CF0A3E52DF2
:10470100F09080017420F0AF2DAE2CAD2BAC2A902F
:074711006FF4122C0DAF291B
:01471800227E
:104079009081E0E0F5280528052805280528052868
:1040890005280528052805280528908010E0F52B26
:10409900A3E0F52CA3E0F52DA3E0F52E9081E1E056
:1040A900F5280528052805280528052805280528AF
:1040B900052805280528908014E0F52FA3E0F530A0
:1040C900A3E0F531A3E0F532E531B52D08E532B5C8
:1040D9002E037F0022E4F528E531540744E0F583F7
:1040E90085328263A201906BB763A2017F08123700
:1040F900DD906BB963A201906AEF63A2017F06129A
:104109003746906BB7E0F529A3E0F52AE4F5289046
:104119006BB7E0702AA3E024F8F528E53154074489
:10412900E0F58385328274082582F582E43583F5CA
:104139008363A201906BB763A201AF281237DDAE8A
:1041490029E4FCFDE532252AF532E5313EF531ED6C
:104159003530F530EC352FF52F908014E52FF0A38D
:10416900E530F0A3E531F0A3E532F090800074402A
:03417900F0AF287C
:01417C002220
:103B54009081E6E0F528052805280528052805288C
:103B640005280528052805280528908028E0F52B38
:103B7400A3E0F52CA3E0F52DA3E0F52E9081E7E07A
:103B8400F5280528052805280528052805280528D9
:103B940005280528052890802CE0F52FA3E0F530B2
:103BA400A3E0F531A3E0F532E4F528E531B52D0ABB
:103BB400E532B52E05C21B023CAEE531540744F094
:103BC400F58385328263A201906BB763A2017F08FB
:103BD4001237DD906BB7E0F529A3E0F52AE52A4515
:103BE4002970099080027410F07F0022906EC3E067
:103BF400FFF4602D906BB9E06F7076906EC4E0FFB7
:103C0400906BBAE06F706A906EC5E0FF906BBBE09A
:103C14006F705E906EC6E0FF906BBCE06F602280B8
:103C240050906BB9E0906EC3F0906BBAE0906EC4A4
:103C3400F0906BBBE0906EC5F0906BBCE0906EC6EC
:103C4400F0906BB7E0702AA3E024F8F528E531542E
:103C54000744F0F58385328274082582F582E435C1
:103C640083F58363A201906BB763A201AF28123777
:103C7400DDAE29E4FCFDE532252AF532E5313EF5D9
:103C840031ED3530F530EC352FF52FAF2EAE2DADAF
:103C94002CAC2BAB32AA31A930A82FD3122BFC4069
:103CA400099080027410F07F002290802CE52FF0A0
:103CB400A3E530F0A3E531F0A3E532F0908002747F
:043CC40040F0AF28F5
:013CC80022D9
:103CC9009081E3E0F5280528052805280528052819
:103CD9000528052805280528052890801CE0F52BCE
:103CE900A3E0F52CA3E0F52DA3E0F52E9081E4E007
:103CF900F528052805280528052805280528052863
:103D0900052805280528908020E0F52FA3E0F53047
:103D1900A3E0F531A3E0F532E4F528E531B52D0A44
:103D2900E532B52E05C21C023E14E531540744E8BC
:103D3900F58385328263A20190684363A2017F0EF5
:103D49001237F3906843E0F529A3E0F52A90684B10
:103D5900E0FFF46045906EBCE0FEEF6E706EA3E08C
:103D6900FF90684CE06F7064906EBEE0FF90684D04
:103D7900E06F7058906EBFE0FF90684EE06F704C36
:103D8900906EC0E0FF90684FE06F7040906EC1E0A8
:103D9900FF906850E06F60048032D28D906843E0F4
:103DA900702AA3E024F2F528E531540744E8F583A5
:103DB900853282740E2582F582E43583F58363A208
:103DC9000190684363A201AF281237F3AE29E4FCDE
:103DD900FDE532252AF532E5313EF531ED3530F58F
:103DE90030EC352FF52FAF2EAE2DAD2CAC2BAB32E1
:103DF900AA31A930A82FD3122BFC5006E52A452950
:103E090070099080017410F07F0022908020E52FC6
:103E1900F0A3E530F0A3E531F0A3E532F09080019D
:053E29007440F0AF2819
:013E2E002271
:044263008E2E8F2FDD
:10426700906FECE0FCA3E0FDA3E0FEA3E0F5358E44
:10427700348D338C32E535FFE5345407FEE42FF5F2
:1042870031EE34C0F530853182F5837423F0053182
:10429700E531700205305330C7F582853083740AE3
:1042A700F00531E531700205305330C7906B8063FC
:1042B700A20185308385318263A2017F061237AF61
:1042C70074062531F531E43530F530852E83852F99
:1042D7008263A20185308385318263A201123793FD
:1042E700908000E020E5F9E4FCFDFE906FECE0F83B
:1042F700A3E0F9A3E0FAA3E02FFFEE3AFEED39FDC4
:10430700EC38FCEF2408FFE43EFEE43DFDE43CFC12
:10431700906FEC122C0D906FECE0908040F0906F56
:10432700EDE0908041F0906FEEE0908042F0906F6A
:0C433700EFE0908043F09080007420F0D4
:014343002257
:06441E008E2E8F2F8D3061
:10442400906FECE0FCA3E0FDA3E0FEA3E0F5368E84
:10443400358D348C33E536FFE5355407FEE42FF52E
:1044440032EE34C0F531853282F5837423F00532BF
:10445400E532700205315331C7F582853183EBF0C3
:104464000532E532700205315331C7906B8063A287
:104474000185318385328263A2017F061237AF74CE
:10448400062532F532E43531F531852E83852F82C8
:1044940063A20185318385328263A201AF30123772
:1044A400AF908000E020E5F974082530F530FFE492
:1044B400FCFDFEE5362FF536EE3535F535ED3534B4
:1044C400F534EC3533F533908040E533F0A3E5342F
:1044D400F0A3E535F0A3E536F09080007420F0AF4A
:0D44E40036AE35AD34AC33906FEC122C0DBC
:0144F10022A8
:0249C6008F411F
:1049C800906FECE0FCA3E0FDA3E0FEA3E0F5458ECC
:1049D800448D438C42E545FFE5445407FEE42FFF30
:1049E800EE34C0906AF663A201F5838F8263A20158
:1049F800AF411237AF908000E020E5F9E4FCFDFEFE
:104A0800E5452541F545EE3544F544ED3543F54397
:104A1800EC3542F542908040E542F0A3E543F0A32F
:104A2800E544F0A3E545F09080007420F0AF45AE72
:0B4A380044AD43AC42906FEC122C0D1B
:014A43002250
:064344008E2D8F2EAB054B
:10434A00906FECE0FCA3E0FDA3E0FEA3E0F5348E61
:10435A00338D328C31E534FFE5335407FEE42FF513
:10436A0030EE34C0F52F853082F5837423F00530A2
:10437A00E5307002052F532FC7F582852F83EBF0A6
:10438A000530E5307002052F906B8063A201852FFE
:10439A008385308263A2017F061237AF7406253007
:1043AA00F530E4352FF52F532FC7E52D853082855B
:1043BA002F83F00530E5307002052F532FC7F582A1
:1043CA00852F83E52EF00530E5307002052F532F37
:1043DA00C7908000E020E5F9E534240AF534E43595
:1043EA0033F533E43532F532E43531F53190804036
:1043FA00E531F0A3E532F0A3E533F0A3E534F0901C
:10440A0080007420F0AF34AE33AD32AC31906FEC33
:03441A00122C0D54
:01441D00227C
:10515400E5D220E0FBC2AF438E2075D2028F828E4F
:0B51640083E0FFE4F5D2538EDFD2AFF2
:01516F00221D
:10518A00E5D220E0FBC2AF43D2028F828E83EDF0DC
:09519A0075D25063D250D2AF224D
:104A4400E4FDED2401FFE433FE12515474782DF596
:104A540082E4346BF583EFF00DBD3FE6E4FDED2415
:104A64007FFFE433FE125154746E2DF582E43469F1
:104A7400F583EFF0746E2DF582E43469F583E0700C
:104A84001B746E2DF582E43469F5837420F0746F21
:104A94002DF582E43469F583E4F080040DBD80BE15
:104AA400E49069EDF0FDEDFF7E0012515474EE2D9B
:0D4AB400F582E43469F583EFF00DBDFEE9F5
:014AC10022D2
:025018008B2DDE
:10501A00A2AF9222C2AF85A22E53A2FE8E838F82A6
:10502A0005A28C838D82740912380BE52D53A2FEDA
:10503A0043A22012380D53A2DF852EA2A22292AFDC
:01504A00FF66
:01504B002242
:10513700A2AF9222C2AF8C838D82EF12380B43A2AB
:0C5147002012380D53A2DFA22292AFFF0D
:015153002239
:0250CB008F282C
:1050CD00A2AF9222C2AFE4F5838D82740612380B23
:1050DD00E52843A22012380D53A2DFA22292AF7F02
:0150ED0001C1
:0150EE00229F
:0250EF008F2808
:1050F100A2AF9222C2AFE4F5838D82740A12380BFB
:10510100E52843A22012380D53A2DFA22292AF7FDD
:01511100019C
:01511200227A
:10366B00A907E7FFA805EF93C3966008403B74FCDE
:10367B002FFF80F00F08EF93C3966008402B74FB6D
:10368B002FFF80E00F08EF93C3966008401B74FA7E
:10369B002FFF80D00F08EF93D3966008400B74F97F
:1036AB002FFF80C01F1F1F1F1FEF54FEF80303F7D0
:1036BB00E893FC08E893FD08E893FE08E893FF22E3
:1036CB0009E993C39D6008402974FB29F980F1092E
:1036DB00E993C39E6008401A74FA29F980E209E95C
:1036EB0093D39F6008400B74F929F980D3191919EA
:1036FB001919E9C313C313FF22740093F8ECC39891
:10370B004024701F740193F8EDC398401970147422
:0E371B000293F8EEC398400E7009740393F801
:10372900EFC39840037F00227F0122EDF8E6F008FD
:10373900A3DFFA22EDF8E0F608A3DFFA22E0A3639B
:10374900A201F0A363A201DFF475A20022E0A36342
:10375900A201F0A363A201E0A363A201F0A363A203
:1037690001E463A201F0A363A201DFE175A20022D3
:10377900E0A363A2016DFE936CFDEE058393FC1536
:103789008363A201DFEA75A200227F00E493A363A9
:10379900A201F00F600CA3E583C2E3F58363A201E4
:1037A90080EA75A20022E0A363A201F0A3E583C227
:1037B900E3F58363A201DFEE75A20022E0A363A211
:1037C90001F0A3E583C2E4D2E3F58363A201DFEC50
:1037D90075A20022E583C2E3F583E0A363A201F0A9
:1037E900A363A201DFEE75A20022E583C2E4D2E35E
:1037F900F583E0A363A201F0A363A201DFEC75A244
:103809000022F922C002C004C00612FFF0D006D07F
:0438190004D00222B3
:104C31000A536572763A00205544502054696D65D7
:104C41004750530A00200A444154414752414D3ACA
:104C510020002043414E2054696D654750530A009E
:104C610020547261737353656E644552520A002079
:104C71005265496E69742043414E0A002043414EFA
:104C8100283029203E20544F210A0020545520303D
:094C91000A0020545520310A00EC
:03001E00E4FF22DA
:10507F00C28DC2AF438901C28C906EE2E0FF700710
:10508F00F58A758CEE800AEFB40A06E4F58A758C02
:06509F0070D28CD2AF229A
:10504C00C28DC2AF438901C28C906EE2E0FF701436
:10505C00302F09F58A758CDCC22F8012758A667523
:10506C008CFC800AEFB40A06E4F58A758CDCD28CD1
:03507C00D2AF228E
:1050A500C230906EE2E0C394645006124C9A1250DE
:1050B5007F12521CD22EE4F558906FEAF0F546F5B2
:0650C5005CC22FF55A2227
:104F6400EF24FCF528201D127E4C7F311242637E13
:104F74006B7FBBE4FBAD2812441E906BBAE0B41FF8
:104F840003D23022906BBB63A201906F6A63A201CB
:0D4F9400AF28123746852846E4F557C22C99
:014FA10022ED
:0F51E200D3EF6480948E5006E55C70028F5C22E0
:10276900208D0302286FC28C202E0302296CE55CA0
:1027790060519068437D48FF12373DE54864017018
:102789001E90684BE0B4FF0ED231201D127E4C7FA3
:10279900381242638009303106E4F55C02296C1273
:1027A900507F124D62201D077E4C7F4612426320E6
:1027B9001D0B7E687F43E4FBAD5C12441EE4F55CAF
:1027C90002296CE546605C746E2557F582E4346F26
:1027D900F583E02405F528D3940E4008E4F546D2A4
:1027E9002C02296C746A2557F582E4346FF5837DD0
:1027F90048AF2812373DE5282557F557E54830E712
:1028090002D22FE548B4010320310612507F124D40
:1028190062E557C39546500302296CE4F546D22C6C
:1028290002296CE5596023906ECE7D48FF12373D31
:10283900E548B40109303106E4F55902296C125012
:102849007F124D62E4F55902296C200216E55BC33B
:102859009464400320160C906EE2E0C39464500324
:10286900124DC412507F123E2F8F28EF7003022998
:102879006C12504CE4F55AE548B4010CD231201DD4
:10288900077E4C7F53124263E55BC3946E4003029B
:102899002943201603022943303075E54864427004
:1028A9006FE54C7032E54AC454F0FFE54BC4540F50
:1028B9002FF548E54BC454F0F549754A0874E325EA
:1028C9005BF582E4346EF5837403255BF55B7D4823
:1028D9007F03123734806374E3255BF582E4346E39
:1028E900F583E528255BF55B7D48AF281237343041
:1028F9001F48C3E55B9528FFE49400FE74E32FF5B8
:1029090082746E3EAF82FEE4FBAD2812441E802A1B
:10291900E548B4420DE54BB40208906AF5E064015C
:10292900601874E3255BF582E4346EF583E52825A8
:102939005BF55B7D48AF28123734301421E5482018
:10294900E71C906DBA7D48AF28123734AF2812467C
:102959006FEF700A201D077E4C7F61124263AF281A
:10296900122D4B30201A301315906EE2E0C3946497
:10297900500C055AE55A94F04004C2AF80FEC220BB
:10298900201503022A81E5586031D39401400415CA
:10299900588028906FEAE004F0E0D39403400D20BA
:1029A9001D077E4C7F701242631250A5201D077EC1
:1029B9004C7F7D124263E4F558D22E302D43E55900
:1029C900703F906ECE04F0A37408F0A37480F0A356
:1029D9007401F0A37406F0906F65E0906ED3F090E7
:1029E9006F66E0906ED4F0906F67E0906ED5F090CE
:1029F9006F68E0906ED6F0E4A3F0A3F075590BC2AE
:102A09002D302B72906F63E07035E5597031906EFF
:102A1900CE7442F0A37408F0906F64E0906ED0F029
:102A2900906F69E0906ED1F0A37401F0755906209A
:102A39001D077E4C7F8C124263906F63E004F09017
:102A49006F63E06402702FE559702B906ECE7402AB
:102A5900F0A37408F0906F64E0906ED0F0A3F0A337
:102A69007401F0755906201D077E4C7F931242634D
:0B2A7900906F63E004F0C2151200260D
:012A8400222F
:104FA200E55B6037E4906CB7F0A3E55BF0906EBB15
:104FB200E0906CB9F0303006A3741FF08006906C5C
:104FC200BA7419F0906EE363A201906CBB63A20104
:0E4FD200AF5B123746E4F55B7F01227F0022C1
:0B51F100302C05C22C7F01227F002221
:0100210022BC
:06521600E4F55BF5462201
:0A51FC00E4906946F0A3F0A3F0224E
:105113002043616E457247495400200A00204361D1
:105123006E457272434821000A000A205265714598
:045133007272210073
:103E2F00E59B541F6020201D1A7E517F13124263A1
:103E3F00E59B541FFF7E007D031243447E517F1D7F
:103E4F00124263E4F59BE5BA30E010E4F5B375B1C7
:103E5F0080F5B2D22EF558906FEAF0E5CFF47003EB
:103E6F00023F60752A01E4F529E5CFF4552A700366
:103E7F00023F4EE529C454F0F5B1E5B2547F6420FA
:103E8F006003023F1FE5B3540FF54C85BC48E5BDF9
:103E9F00541FFF131313541FFFE5BD54E044184F75
:103EAF00F549E5BDC43354E0FFE5BE131313541FAA
:103EBF004FF54AE5BEC43354E0FFE5BF1313135467
:103ECF001F4FF54B85A34D85A34E85A34F85A3505B
:103EDF0085A35185A35285A35385A354E4F5B2203E
:103EEF00020CE548547EB5480575B350800375B391
:103EFF00D0E54C700AE548547EB548037F00223068
:103F0F000208E54830E7037F0022E54C2405FF2235
:103F1F00E5B2549F6023201D207E517F2012426303
:103F2F00AFB27E007D03124344AFB37E007D031218
:103F3F0043447E517F2B124263E4F5B275B3D0E553
:103F4F002A25E0F52A0529E529C394085003023EE6
:033F5F00787F0068
:013F6200223C
:104D6200906EE2E0C39464505675B180E4F5B3F5F9
:104D7200B28548BCE54AC4135407FFE54954E04FE5
:104D8200F5BDE54A33333354F8FFE54BC4135407FA
:104D92004FF5BEE54B33333354F8F5BF854DA3854C
:104DA2004EA3854FA38550A38551A38552A3855356
:104DB200A38554A3E54C540F2450F5B375580AC289
:024DC2002E229F
:104DC40075B190E5B220E613201D107E517F2D129F
:104DD4004263AFB27E007D03124344E4F5B3F5B2FF
:104DE40074892515F582E43461F583E0F5BCE4F5B6
:104DF400BD748A2515F582E43461F583E0FF33330D
:104E04003354F8F5BE75BF78051505157489251555
:104E1400F582E43461F583E07002F51575B3502230
:09520600EF6003C29622D2962249
:104C9A0043AB01C2E8C2EAE4FFEFC454F0F5B1C382
:104CAA00EF64809488500575B3D08003E4F5B3E4CB
:104CBA00F5B2F5BCF5BDF5BEF5BFF5C4F5C5F5C64B
:104CCA00F5C7F5A3F5A3F5A3F5A3F5A3F5A3F5A3F6
:104CDA00F5A30FBF0EC3906EE2E0FF25E0F5B475B1
:104CEA00B50C75B66C75A11275AB0275C13E75C36C
:044CFA00FF75C2037D
:014CFE002293
:10125D005452414E5A004D4158420052545300448D
:10126D00454C4159004D4F4445004B5000545500DD
:10127D0043414E004B5654004154004449520043E3
:10128D00414E4D4F4E00475254494D45005449541F
:10129D0053005453494E5600003E2A2C312CCFE0BA
:1012AD00F0E0ECE5F2F0FB20F3EFF0E0E2EBFFFE17
:1012BD00F9E5E3EE20EAEEEDF2F0EEEBEBE5F0E032
:1012CD0020CACF20C8F1E5F2FC0A003E4C2C6B3051
:1012DD00312C25732C43EAEEF0EEF1F2FC20EDE01B
:1012ED0020F8E8EDE52043414E2C30202D203530FF
:1012FD0030EAE1283530EC292C31202D203530EA2B
:10130D00E128353030EC290A0030202D20353030E1
:10131D00EAE1283530EC290031202D203530EAE185
:10132D0028353030EC29003E532C6B30322C2562A1
:10133D00752CCCE0EAF12E20E0E4F0E5F120E1EBB4
:10134D00EEEAE020D2D128302D38290A003E532C68
:10135D006B30332C2562752CCCE0EAF12E20E0E4C5
:10136D00F0E5F120E1EBEEEAE020D2C8D228302DF5
:10137D0038290A003E532C6B30342C2562752CCC49
:10138D00E0EAF12E20E0E4F0E5F120E1EBEEEAE019
:10139D0020D2D328302D38290A003E422C6330311B
:1013AD002C2562752CC2F2EEF0E8F7EDFBE920EA90
:1013BD00EEEDF2F0EEEBEBE5F020EDE020F8E8EDF0
:1013CD00E50A003E2A2C312CCFE0F0E0ECE5F2F0FE
:1013DD00FB20EFF0EEF2EEEAEEEBE020C3F0E0EDF5
:1013ED00E8F220EFEE20EFEEF0F2F320525332331D
:1013FD00320A003E4C2C6B30352C256C752CD1EA05
:10140D00EEF0EEF1F2FC20EEE1ECE5EDE020EDE0AA
:10141D0020EFEEF0F2F32C3130302C3230302C3313
:10142D0030302C3630302C313230302C32343030AC
:10143D002C343830302C393630302C313932303084
:10144D002C33383430302C35373630302C31313573
:10145D003230300A003E532C6B30362C2562752C01
:10146D00CDEEECE5F020CACF200A003E422C6730CD
:10147D00312C2562752CCCE0E3E8F1F2F0E0EBFCC9
:10148D000A003E422C6730322C2562752CC8EDE2E5
:10149D00E5F0F2E8F0EEE2E0F2FC20E7EDE0F7E552
:1014AD00EDE8FF20D2D10A003E422C6730332C25C7
:1014BD0062752CC8F1EFEEEBFCE7EEE2E0F2FC20FA
:1014CD00F0E0F1F8E8F0E5EDEDFBE920EFF0EEF2FC
:1014DD00EEEAEEEB20F1EE20E2F0E5ECE5EDE5ECE9
:1014ED000A003E422C6730342C2562752CC2FBF16C
:1014FD00F2E0E2EBFFF2FC2052545320EFF0E82033
:10150D00EFE5F0E5E4E0F7E50A003E532C673035F2
:10151D002C2562752CC7E0E4E5F0E6EAE020EFE566
:10152D00F0E5E4E0F7E820EFEEF1EBE5205254535F
:10153D0020282A3130ECF1290A003E532C67303631
:10154D002C2562752C4BEEECECF3F2E8F0F3E5ECA8
:10155D00E0FF20EBE8EDE8E820F1E2FFE7E82028E6
:10156D0030290A003C21003C6B30313D003C6B3092
:10157D00323D003C6B30333D003C6B30343D003C24
:10158D006330313D003C6B30353D003C6B30363DBA
:10159D00003C6730313D003C6730323D003C6730E8
:1015AD00333D003C6730343D003C6730353D003CF9
:1015BD006730363D000A41734F55543A2000544967
:1015CD0049204379636C650A005453204379636C59
:1015DD00650A0054530A005455204F4B0A005455C8
:1015ED0020446961670A005455205265710A002034
:1015FD0054552054696D654F5554210A004154636B
:10160D006F6E6E6563740A000A4173494E3A20008D
:10161D000A435243204552523A20000A4E6B703A0B
:10162D0020000ACFF0E8EDFFF2E020EAEEECE0ED6D
:10163D00E4E020D2D320002020D2D320E7E0EDFF3C
:10164D00F2EE210A000ACDE520EFEEEDFFEB20F2E0
:10165D00E8EF20EFE0EAE5F2E0210A000011233285
:10166D00465765748C9DAFBECADBE9F81001332275
:10167D00564775649C8DBFAEDACBF9E82130021365
:10168D0067764455ADBC8E9FEBFAC8D93120120355
:10169D0077665445BDAC9E8FFBEAD8C94253617045
:1016AD0004152736CEDFEDFC8899ABBA5243716035
:1016BD0014053726DECFFDEC9889BBAA6372405125
:1016CD0025340617EFFECCDDA9B88A9B7362504115
:1016DD0035241607FFEEDCCDB9A89A8B8495A7B6F5
:1016ED00C2D3E1F008192B3A4E5F6D7C9485B7A6F5
:1016FD00D2C3F1E018093B2A5E4F7D6CA5B48697E5
:10170D00E3F2C0D129380A1B6F7E4C5DB5A49687D4
:10171D00F3E2D0C139281A0B7F6E5C4DC6D7E5F4C4
:10172D008091A3B24A5B69780C1D2F3ED6C7F5E4B4
:10173D009081B3A25A4B79681C0D3F2EE7F6C4D5A4
:10174D00A1B082936B7A48592D3C0E1FF7E6D4C594
:10175D00B1A092837B6A58493D2C1E0F0089129BC4
:10176D0024AD36BF48C15AD36CE57EF78108931A74
:10177D00A52CB73EC940DB52ED64FF76028B109964
:10178D0026AF34BD4AC358D16EE77CF5830A911854
:10179D00A72EB53CCB42D950EF66FD74048D169F34
:1017AD0020A932BB4CC55ED768E17AF3850C971E34
:1017BD00A128B33ACD44DF56E960FB72068F149D24
:1017CD0022AB30B94EC75CD56AE378F1870E951C14
:1017DD00A32AB138CF46DD54EB62F97008811A9314
:1017ED002CA53EB740C952DB64ED76FF89009B12F4
:1017FD00AD24BF36C148D35AE56CF77E0A831891E4
:10180D002EA73CB542CB50D966EF74FD8B029910D3
:10181D00AF26BD34C34AD158E76EF57C0C851E97B3
:10182D0028A13AB344CD56DF60E972FB8D049F16B3
:10183D00A920BB32C54CD75EE168F37A0E871C95A3
:10184D002AA338B146CF54DD62EB70F98F069D1493
:10185D00AB22B930C74ED55CE36AF1780008040CB1
:10186D00020A060E0109050D030B070FFF125DFF9E
:10187D001263FF1268FF126CFF1272FF1277FF12D4
:10188D007AFF127DFF1281FF1285FF1288FF128CE5
:0C189D00FF1293FF129AFF129FFF12A58A
:1051BA00EF540F90186993FEC454F0FEEFC4540FD5
:0451CA00932EFF22FF
:030023000244F2A2
:0B44F200C0E0C083C082C0D075D018AD
:1044FD00309852C298756001AF9920074820030B80
:10450D00EF64027040D203D291803A300C04C20C99
:10451D008024BF0904D20C802CBF0205530C80806F
:10452D0024BF0312906616E50CF0630C80530C80CB
:10453D00C203C291800F7439250CF582E43466F5FF
:10454D0083EFF0050C30995F30045A906187E0FFDE
:10455D00E50DC39F4008C204D211C2908047D2908E
:10456D00AF0D050D74392FF582E43467F583E0F551
:10457D0010300B1953107F30012830D0083006222F
:10458D00631080801D20061A631080801530011283
:10459D00E50B5210300606A2D0929B8005A2D0B337
:0745AD00929B851099C29951
:0945B400D0D0D082D083D0E032D7
:103F63007BFF7A1279A612246F906EE2E0701475CB
:103F730030FF7531137532167BFF7A1279D812240C
:103F83006F80127530FF7531137532257BFF7A12FE
:103F930079D812246F7BFF7A137934906188E0F526
:103FA3003012246F7BFF7A13795A906101E0F53068
:103FB30012246F7BFF7A137981906100E0F5301250
:103FC300246F7BFF7A1379A7A202E433F53012241E
:103FD3006F7BFF7A1379D012246F90683DE0FEA3C4
:103FE300E0FFC3E49FFFE49EFEAB07FA3395E0F9DD
:103FF300F87F007E8C7D0A7C00122B5C8F338E321F
:104003008D318C307BFF7A14790012246F7BFF7A19
:10401300147962906405E0F53012246F7BFF7A1403
:10402300797890683BE06401F53012246F7BFF7A66
:1040330014798FA20AE433F53012246F7BFF7A14CC
:1040430079B5A205E433F53012246F7BFF7A147936
:10405300EFA20FE433F53012246F7BFF7A15791743
:1040630085093012246F7BFF7A15794790683AE00F
:06407300F53012246F225B
:1039C1007E157F7112483BEF4E70037F0122E49018
:1039D1006EE2F07E157F7412483BEF4E6015125176
:1039E10070BF3106906EE2740AF0BF3206906EE24B
:1039F1007464F07E157F7A12483BEF4E600A124ED6
:103A010024906188EFF080069061887402F07E1541
:103A11007F8012483BEF4E600A124E24906101EF05
:103A2100F080069061017402F07E157F8612483B9A
:103A3100EF4E600A124E24906100EFF08006906113
:103A4100007402F07E157F8C12483BEF4E600D1220
:103A51004E24EC4D4E4F24FF92028002C2027E158D
:103A61007F9212483BEF4E6023124E24A804A90511
:103A7100AA06AB077F007E8C7D0A7C00122B5C12AC
:103A81002BEE90683DEEF0A3EFF0800A90683D7454
:103A9100FFF0A374DCF07E157F9812483BEF4E6077
:103AA1000A124E24906405EFF080069064057401BB
:103AB100F07E157F9E12483BEF4E600E125170EF63
:103AC10024D0640190683BF08005E490683BF07E6F
:103AD100157FA412483BEF4E600C125170EF24D0B9
:103AE10024FF920A8002C20A7E157FAA12483BEF88
:103AF1004E600C125170EF24D024FF92058002C257
:103B0100057E157FB012483BEF4E600C125170EFED
:103B110024D024FF920F8002C20F7E157FB6124877
:103B21003BEF4E6007124E248F098003E4F5097EB6
:103B3100157FBC12483BEF4E600D124E2490683940
:103B4100EEF0A3EFF08009906839E4F0A37478F007
:023B51007F00F3
:013B5300224F
:10300400E4F528E52875F003A42479F582E434185E
:10301400F583E493FB740193FA740293F9122A85FD
:10302400700302328EE4F52AF52BF529746E2529F6
:10303400F582E43469F583E0FF7003023289E52800
:1030440075F003A42479F582E43418F583E493FB42
:10305400740193FA740293F9852A82758300122A03
:103064009EFEEFB50608752B01052A023284E52B76
:103074007003023284EE600302327FE528B40F004D
:103084004003023289903090F82828730230BD0240
:10309400310402313D02314202316D0231CF02323C
:1030A400890231A10232890231FD023246023273B1
:1030B40002327702328902327B746E2529F9E434B4
:1030C40069FA7B01C0031B8B33753400753500E44A
:1030D400F536D00312381D8F2F8E2E8D2D8C2CABF0
:1030E4002FAA2EA92DA82C7F007E8C7D0A7C00128D
:1030F4002B5C122BEE90683DEEF0A3EFF0023289C8
:10310400746E2529F582E43469F583E024D0906156
:1031140088F0746F2529F582E43469F583E024D0BE
:10312400906101F074702529F582E43469F583E037
:1031340024D0906100F0023289D20F023289746E79
:103144002529F9E43469FA7B01C0031B8B337534F8
:1031540000753500E4F536D00312381D8F2F8E2EFE
:103164008D2D8C2C8F09023289746E2529F582E409
:103174003469F583E0B43702D20B746F2529F582E4
:10318400E43469F583E0FFB44E04C2018002D20145
:10319400EF64456003023289D206023289746E25D7
:1031A40029F9E43469FA7B01C0031B8B33753400BD
:1031B400753500E4F536D00312381D8F2F8E2E8D11
:1031C4002D8C2C906EE2EFF0023289746E2529F971
:1031D400E43469FA7B01C0031B8B33753400753505
:1031E40000E4F536D00312381D8F2F8E2E8D2D8CD2
:1031F4002C906405EFF0023289746E2529F9E434C9
:1032040069FA7B01C0031B8B33753400753500E408
:10321400F536D00312381D8F2F8E2E8D2D8C2CE475
:10322400FFFEFDFCAB2FAA2EA92DA82CD3122BFC3C
:10323400400A906839E52EF0A3E52FF0D20EC20DB6
:103244008043746E2529F9E43469FA7B01C0031BB9
:103254008B33753400753500E4F536D00312381D10
:103264008F2F8E2E8D2D8C2C90683BEFF08016D2F4
:10327400028012D205800EC20A800AE4F52BF52AD8
:0A328400052902303005280230074A
:01328E00221D
:10348200C22BC210C209C208906184740AF0E4908F
:10349200683CF090683AE024F9FE906839E034FF25
:1034A200906303F0A3CEF0E4906186F0C2129066BE
:1034B200187405F0C22DE4F508906944E064557073
:1034C20004A3E06481603BE4FF7F409061B9E4F0D3
:1034D200A3DFFCE4FF7F20906619E4F0A3DFFCE4A5
:1034E200FF74062FF582E43466F583E4F0740E2F40
:1034F200F582E43466F583E4F00FBF08E4E4F50EE8
:10350200F50FE4F514F513906302F0906301F0C235
:1035120004C211C207C203C20CF50D906187F0F517
:1035220009F50CF560C200C20BC20F90683D74FF32
:10353200F0A374F4F0750BFFC20EE4906405F090F2
:10354200683BF0D20DC202C205906839F0A37478CC
:10355200F0D20AE4906EE2F01239C1EF6003123049
:1035620004E4F5157E617F89906188E0F515E51523
:10357200C394014007E515D394084003E4F515E52B
:103582001560220FEFAC0670010E14F5828C837465
:10359200C4F015150FEFAC0670010E14F5828C8382
:1035A200E515F080DA906101E0F515E515C39401A7
:1035B2004007E515D394084003E4F515E5156022AC
:1035C2000FEFAC0670010E14F5828C8374C8F015EF
:1035D200150FEFAC0670010E14F5828C83E515F021
:1035E20080DA906100E0F515E515C394014007E526
:1035F20015D394084003E4F515E51560220FEFACEE
:103602000670010E14F5828C8374C2F015150FEF4B
:10361200AC0670010E14F5828C83E515F080DA0F8A
:10362200EFAC0670010E14F5828C83E4F08F828E6B
:1036320083F0F515C2ADF5C9D2CDD2CCC2C9C2CA8A
:10364200F5CDF5CC90683DE0F5CBA3E0F5CA85CB8E
:10365200CD85CACCD29ED29CD2CAC2ACC298C299E3
:0836620075B81075B710D2AC69
:01366A00223D
:1051CE00E5126FFF901769936511F512EF9016694E
:0351DE0093F51135
:0151E10022AB
:0245BD008F2E3F
:1045BF00E4FC752F61753002F512F511FDEDC39511
:1045CF002E50170530E530AE2F7002052F14F582EF
:1045DF008E83E0FF1251CE0D80E30530E530AE2F14
:1045EF007002052F14F5828E83E512F085308285D7
:1045FF002F83E511F0052E052E7E677F39752F610C
:10460F007530028F828E837402F00FBF00010E0C83
:10461F00E4FDEDC3952E5038853082852F83E0F968
:10462F0064026008E964036003B9090D8F828E8309
:10463F007409F00FBF00010E0C8F828E83E9F00F0B
:10464F00BF00010E0C0530E5307002052F0D80C242
:0F465F008F828E837403F00FBF00010E0CAF0427
:01466E002229
:03521C00C20722A4
:104F21008F2D20043D300D3AAF2D1245BD90618784
:104F3100EFF0201D127E157FC21242637E617F0257
:104F4100E4FBAD2D12441E300F057F01125206E520
:104F5100096003F55D22E4F50DD204C2992099FDA3
:034F6100D29922C0
:022D4B008F29CE
:102D4D00906405E07003023003E54824BE70030271
:102D5D002FAC24FA7003022F3024046003023003D9
:102D6D00E54930E703022E1B201D077E157FCB1290
:102D7D004263E54B6068E54AC394024003023003A9
:102D8D00E54A7007E54B14F52A8006E54B241FF53F
:102D9D002AE52A75F004A42405F582746335F0F54F
:102DAD00837D4D7F04123734E52A75F004A4240188
:102DBD00F582746235F0F5837D517F0412373474DA
:102DCD00F9254AF582E43461F5837481F074B925EF
:102DDD002AF582E43461F5837401F0D20822201DB6
:102DED00077E157FD61242637406254AF582E434B8
:102DFD0066F5837480F0E54A75F004A42419F58214
:102E0D00746635F0F5837D4D7F0412373422E54C21
:102E1D0064086003023003E54AC3940440030230A2
:102E2D0003201D077E157FE0124263752901E54BD6
:102E3D005407FFE529A807088002C333D8FCF529FC
:102E4D007408250FF50FB50E067408250EF50EE561
:102E5D004B547FFFE54AC43354E02FFE7400250F19
:102E6D00F582E43460F583EEF0E54BC39480502297
:102E7D00EF131313541FFFE54A25E025E02F241906
:102E8D00F582E43466F583E0FFE529F4FEEF5EF0AC
:102E9D00802EE54B547FFF131313541FFFE54A2576
:102EAD00E025E02F2419F582E43466F583E0452909
:102EBD00F07400250FF582E43460F583E04480F072
:102ECD007401250FF582E43460F5837D4D7F041286
:102EDD003734E552FEE551FF7C007D0A122ACBEF17
:102EED007405250FF582E43460F583EFF074062543
:102EFD000FF582E43460F583E553F07407250FF583
:102F0D0082E43460F583E554F0301D030230037420
:102F1D0000250FF582E43460AF82FEE4FB7D0812DC
:102F2D00441E22E54B54E064407003023003E54A31
:102F3D00701DE54B1313543FFF7401A80708800261
:102F4D00C333D8FC4213906301E04513F08024E5B0
:102F5D004A64016003023003E54B1313543FFF74C1
:102F6D0001A807088002C333D8FC4214906302E025
:102F7D004514F0E54A75F020A4FFE54B547F7C0025
:102F8D002FFFEC35F0FEEF25E0FFEE33FE74062F3C
:102F9D00F58274643EF5837D4DAF4C12373422E5D6
:102FAD004BB40113201D077E157FE4124263E54EDD
:102FBD0004906FEBF0C22BE54BB40216240EF58294
:102FCD00E43466F583E54EF0201D077E157FEB1288
:102FDD004263E54BB4031F240EF582E43466F5839A
:102FED00E54EF0201D077E157FF4124263302B064F
:062FFD00906F637402F006
:0130030022AA
:10002600906405E07003020A19301361050A9066B0
:1000360018E0600214F090683CE0600214F09068EA
:100046003BE06008906184E0600214F0C213300E59
:1000560021906839E0FEA3E0FFD3906304E09F900F
:100066006303E09E500CA3E004F07006906303E087
:1000760004F0302B18906185E004F0E0D3940A4038
:100086000C201D077E157FFC124263C22BE55DB472
:10009600010EE4F55DF50DD204C2992099FDD299C1
:1000A60030040DE50AD394064009C204D211800338
:1000B600E4F50A200E0302019190683AE024FBFF62
:1000C600906839E034FFFEC3906304E09F906303B9
:1000D600E09E4012906186E0700CC20DFF1252063F
:1000E6009061867401F090683AE024FDFF906839CB
:1000F600E034FFFEC3906304E09F906303E09E40FC
:1001060012906186E0B4010B7F011252069061865F
:100116007402F090683AE024FEFF906839E034FFFC
:10012600FEC3906304E09F906303E09E405D20045D
:100136005A9067397441F0A37454F0A37424F0A361
:100146007443F0A3744FF0A314F0A3F0A37445F026
:10015600A37443F0A37454F0A3740DF0A3740AF0CF
:10016600906187740CF0E4F50DD204C2992099FDD4
:10017600D299E4906303F0A3F0906186F0301D03FA
:10018600020A197E167F0A1242632230110AC21130
:10019600300F05E4FF125206300403020678E55DCF
:1001A6006003020678200D03020678906184E06001
:1001B6000302067890683BE06007E4906184F08073
:1001C60006906184740AF0301229C212E49061022A
:1001D600F0A37408F0906405E0906104F09066174F
:1001E600E0906105F0A374FEF0A3748FF07F061211
:1001F6004F2122906FEBE0FF6025E4906102F0A3AF
:100206007408F0906405E0906104F0A37483F0A391
:10021600EFF0E4A3F0906FEBF07F06124F2122E59A
:100226000F650E700302032690683CE0600302042B
:1002360012E50E2408F529E4906102F0A37408F093
:10024600906405E0906104F0A374F0F0A37406F0E6
:10025600A37491F074062529F582E43460F583E0F1
:10026600906108F074072529F582E43460F583E08F
:10027600906109F074012529F582E43460F583E084
:1002860090610AF074022529F582E43460F583E072
:1002960090610BF074032529F582E43460F583E060
:1002A60090610CF074042529F582E43460F583E04E
:1002B60090610DF074002529F582E43460F583E041
:1002C600FF547FFEC39440500BEFC454F00490617A
:1002D6000EF0801674002529F582E43460F583E07B
:1002E600FFC454F0240590610EF074002529F582B0
:1002F600E43460F583E0FFEEC4540F90610FF0EF35
:100306005480FF74052529F582E43460F583E02FD7
:10031600906110F090683C7414F07F0F124F212208
:10032600300973906606E0D39400406AE490610257
:10033600F0A37408F0906405E0906104F0A37441A2
:10034600F0A37420F0752B61752C07E4F529741958
:100356002529F582E43466F583E0F52A300A06FF9E
:100366001251BA8F2A852C82852B83E52AF0F4FF59
:10037600E5822408F582E43583F583EFF0052CE564
:100386002C7002052B0529E529C3940840C07F156A
:10039600124F21C20922301073906607E0D39400F1
:1003A600406AE4906102F0A37408F0906405E0905E
:1003B6006104F0A37445F0A37420F0752B61752CCD
:1003C6000775290874192529F582E43466F583E052
:1003D600F52A300A06FF1251BA8F2A852C82852B00
:1003E60083E52AF0F4FFE5822408F582E43583F5F7
:1003F60083EFF0052CE52C7002052B0529E529C3B2
:10040600941040C07F15124F21C21022200803020B
:1004160005159061FAE0FF9061F9E04F5401D3941D
:10042600005003020515E4F52974B92529F582E47F
:100436003461F583E0700302050774B92529F58256
:10044600E43461F583E4F0906102F0A37408F0905F
:100456006405E0906104F0A374F0F0A37403F0A3C4
:100466007491F0E529C4540F2408A3F0E529540F2C
:10047600A3F0E52925E025E0F5292401F582E434F9
:1004860062F583E090610AF074022529F582E4346E
:1004960062F583E090610BF074032529F582E4345C
:1004A60062F583E090610CF074042529F582E4344A
:1004B60062F583E090610DF0E4A3F074052529F55B
:1004C60082E43463F583E090610FF074062529F524
:1004D60082E43463F583E0906110F074072529F512
:1004E60082E43463F583E0906111F074082529F500
:1004F60082E43463F583E0906112F07F11124F219C
:10050600220529E529C39440500302042FC208900E
:100516006618E0704130053E7478F0E4906102F0B0
:10052600A37408F0906405E0906104F0A374F0F001
:10053600E4A3F0A37490F0A37408F0E4A3F0A3F08E
:10054600A3F0A3F0A3F0A3F0A3F0A3F0A3F0A3F00D
:100556007F11124F2122E508C394045070E5082547
:10056600E0FF7403A807088002C333D8FCF52955B9
:100576001365297053E529F45213E4906102F0A340
:100586007408F0906405E0906104F0A374F0F0A3A1
:100596007402F0A37491F0E5082420A3F0E5083373
:1005A600333354F875F002A42406F582E5F034647A
:1005B600F58363A20190610963A2017F1012374699
:1005C6007F17124F210508220508020653E508C3C6
:1005D60094085076E50824FC25E0FF7403A8070874
:1005E6008002C333D8FCF529551465297058E529CE
:1005F600F45214E4906102F0A37408F0906405E0EC
:10060600906104F0A374F0F0A37402F0A37491F067
:10061600E50854032440A3F0E50833333354F87552
:10062600F002A42406F582E5F03464F58363A201A2
:1006360090610963A2017F101237467F17124F217E
:1006460005085308072205088003E4F50890683B6F
:10065600E0701F906102F0A37408F0906405E090CA
:100666006104F0A37490F0E4A3F0A3F07F06124FA8
:100676002122906616E0FF7003020A19F52AE4F0BB
:10068600201D1F7E167F15124263E52A54802439E9
:10069600F582E43466AF82FEE52A547FFDE4FB1260
:1006A600441EE52A7003020A19E52A5480FF2439FC
:1006B600F582E43466AD82F52B8D2CE4F512F51146
:1006C6008F29E529C3952A5018052CE52CAE2B70E9
:1006D60002052B14F5828E83E0FF1251CE05298088
:1006E600E1E51145126026301D03020A197E167FC8
:1006F6001D124263E52A54802439F582E43466AF3C
:1007060082FEE52A547FFDE4FB12441E22E4906338
:1007160003F0A3F0D20D906186F0E52A54802439C7
:10072600F582E43466AF82F52B8F2C7402252CF506
:100736002CE4352BF52B852C82F583E0FF906405A0
:10074600E0FEEF6E6026301D03020A197E167F2832
:10075600124263E52A54802439F582E43466AF8276
:10076600FEE52A547FFDE4FB12441E22052CE52CEF
:100776007002052BF582852B83E0FFB43006E490EA
:100786006184F022EF64017003020A19EFB41805C0
:10079600D209D21022EFB4190B906301E0F513A32E
:1007A600E0F51422852C82852B83E0FF54F064F05B
:1007B60060030208A1906617EFF0052CE52C700285
:1007C600052BF582852B83E0FF64807033052CE5CD
:1007D6002C7002052BF582852B83E06440600302B2
:1007E6000A19D212052CE52C7002052BF582852BF1
:1007F60083E064086003020A19D205906618F022A5
:10080600EFB40127052CE52C7002052BF582852B0C
:1008160083E0644F6003020A1990683CE0700302AB
:100826000A197408250EF50EE4F022852C82852B14
:1008360083E06003020A19052CE52C7002052BF5EE
:1008460082852B83E064426003020A19052CE52C9D
:100856007002052BF582852B83E0906F65F0052CE1
:10086600E52C7002052BF582852B83E0906F66F0F0
:10087600052CE52C7002052BF582852B83E0906F05
:1008860067F0052CE52C7002052BF582852B83E09D
:10089600906F68F0D22DC205D21222852C82852B4C
:1008A60083E0FF64116008EF641260030209F7E554
:1008B6002A547F640E60030209F7201D077E167F07
:1008C6002F124263302B0E301D03020A197E167F4B
:1008D6004412426322852C82852B83E0540314F54F
:1008E6002A052CE52C7002052BF582852B83E0F575
:1008F6002930E709E4906F64F0906F69F0E52930DC
:10090600E60BE4906F64F0906F697410F0E529309F
:10091600E50B906F647401F0E4906F69F0E529309F
:10092600E40C906F647401F0906F697410F0E5291F
:1009360030E30B906F647402F0E4906F69F0E52980
:1009460030E20C906F647402F0906F697410F0E5F9
:100956002930E10B906F647403F0E4906F69F0E561
:100966002930E00C906F647403F0906F697410F096
:100976007402252CF52CE4352BF52B852C82F5837A
:10098600E0F52930E700E52930E607906F69E024B5
:1009960002F0E52930E507906F69E02404F0E529C7
:1009A60030E407906F69E02406F0E52930E307900C
:1009B6006F69E02408F0E52930E207906F69E024CA
:1009C6000AF0E52930E107906F69E0240CF0E5298B
:1009D60030E007906F69E0240EF0906F69E0252AF9
:1009E600F0D22BE4906185F0906F63F0906FEBF09E
:1009F60022201D1F7E167F52124263E52A54802450
:100A060039F582E43466AF82FEE52A547FFDE4FBC5
:030A160012441E69
:010A190022BA
:1047BB000218A9E493A3F8E493A34003F68001F253
:1047CB0008DFF48029E493A3F85407240CC8C333FF
:1047DB00C4540F4420C8834004F456800146F6DFCE
:1047EB00E4800B010204081020408090520FE47EFD
:1047FB00019360BCA3FF543F30E509541FFEE493C3
:10480B00A360010ECF54C025E060A840B8E493A389
:10481B00FAE493A3F8E493A3C8C582C8CAC583CAB4
:10482B00F0A3C8C582C8CAC583CADFE9DEE780BE6C
:015215000098
:102A8500BB010689828A83E0225002E722BBFE024F
:092A9500E32289828A83E4932282
:102A9E00BB010CE58229F582E5833AF583E02250ED
:102AAE0006E92582F8E622BBFE06E92582F8E22237
:0D2ABE00E58229F582E5833AF583E4932251
:102ACB00BC000BBE0029EF8DF084FFADF022E4CCEF
:102ADB00F875F008EF2FFFEE33FEEC33FCEE9DECB8
:102AEB00984005FCEE9DFE0FD5F0E9E4CEFD22EDFE
:102AFB00F8F5F0EE8420D21CFEADF075F008EF2F48
:102B0B00FFED33FD4007985006D5F0F222C398FD38
:052B1B000FD5F0EA22D5
:102B200075F008758200EF2FFFEE33FECD33CDCC6C
:102B300033CCC58233C5829BED9AEC99E5829840EF
:102B40000CF582EE9BFEED9AFDEC99FC0FD5F0D6CC
:102B5000E4CEFBE4CDFAE4CCF9A88222B800C1B9F6
:102B60000059BA002DEC8BF084CFCECDFCE5F0CB34
:102B7000F97818EF2FFFEE33FEED33FDEC33FCEB6D
:102B800033FB10D703994004EB99FB0FD8E5E4F928
:102B9000FA227818EF2FFFEE33FEED33FDEC33FC15
:102BA000C933C910D7059BE99A4007EC9BFCE99A09
:102BB000F90FD8E0E4C9FAE4CCFB2275F010EF2F4E
:102BC000FFEE33FEED33FDCC33CCC833C810D7074E
:102BD0009BEC9AE899400AED9BFDEC9AFCE899F889
:0E2BE0000FD5F0DAE4CDFBE4CCFAE4C8F9221C
:0E2BEE00C3E49FFFE49EFEE49DFDE49CFC22F8
:102BFC00EB9FF5F0EA9E42F0E99D42F0E89C45F02F
:012C0C0022A5
:0C2C0D00ECF0A3EDF0A3EEF0A3EFF0223A
:102C1900A8828583F0D083D082122C30122C3012F6
:102C29002C30122C30E473E493A3C583C5F0C5831B
:102C3900C8C582C8F0A3C583C5F0C583C8C582C805
:012C49002268
:10240D00E53C2430F8E6053C22782D302902783061
:10241D00E475F001122CAB022A852022EB7F2ED21F
:10242D00228018EF540F2490D43440D4FF30260B63
:10243D00EF24BFB41A0050032461FFE53D6002157F
:10244D003D0540E5407002053F30290D782DE475BE
:10245D00F001122CABEF022C4A024EDA7403D22992
:10246D008003E4C229F53C8B2D8A2E892FE4F53D9E
:10247D00F53FF540E53D60077F2012244880F57556
:10248D003EFFC223C222C224C225C227C228C22AAD
:10249D00122416FF700D3029057F00122459AF400C
:1024AD00AE3F22B4255FC2D5C226122416FF24D01A
:1024BD00B40A00501A75F00A783D30D50508B6FFFC
:1024CD000106C6A426F620D5047002D22580D92493
:1024DD00CFB41A00EF5004C2E5D226022659D223FA
:1024ED0080C6D22280C0D22480BCD2D580BAD22759
:1024FD0080B47F201224482024077401B53D00408C
:10250D00F112240DFF122448022481D22AD22880F0
:10251D009512240DFB12240DFA12240DF94A4B705D
:10252D0006792A7A277BFF20242EE53D602A7E003E
:10253D008E82758300122A9E60060EEE653E70F047
:10254D00C2D5EBC0E0EAC0E0E9C0E0EE1226A0D0B3
:10255D00E0F9D0E0FAD0E0FB122A85FF60AAEBC0CB
:10256D00E0EAC0E0E9C0E0122448D0E02401F9D04F
:10257D00E03400FAD0E0FBE53E0460DCD53ED980C6
:10258D00877BFF7A26799CD224809C7910800279F2
:10259D0008C228C22A8008D2D5790A8004790AC2D5
:1025AD00D5E53E047002F53EE4FAFDFEFF12240D62
:1025BD00FC7B0820231312240DFD7B1030220A1200
:1025CD00240DFE12240DFF7B20EC3382D592D550C5
:1025DD0013C3E43022069FFFE49EFEE42023039DF7
:1025ED00FDE49CFCE4CBF8C223EC700CCFCECDCC3B
:1025FD00E824F8F870F38017C3EF33FFEE33FEEDE8
:10260D0033FDEC33FCEB33FB994002FB0FD8E9EBC8
:10261D00302305F8D0E0C448B223C0E00AEC4D4E9B
:10262D004F78207B0070C2EAB53E0040BCC0E0127E
:10263D0026A2D0F0D0E0202304C4C0E0C4B223C051
:10264D00F0122431D0F0D5F0EB022481122D0A25A1
:10265D001E5325985824EF4C24EB42259C4F25A45E
:0F266D004425A44925044325AA55258E46258ECC
:10267C0045258E47274A5024F32D24F72E251A2B57
:10268C0024FB2325182027332A24B34800002512C5
:10269C003F3F3F00790AA2D5202514302709B910F5
:1026AC00020404B9080104A2D52028025001042018
:1026BC0024689224B53D005034C0E07F20302519A9
:1026CC007F30A22472287227500F1226F9C224C21E
:1026DC0028C227C22A7F30800F302703E9C0E012BE
:1026EC002448302703D0E0F9D0E0B53DCC30271793
:1026FC007F30B9100C1224487F583026077F788021
:10270C0003B908031224483024057F2D0224487F86
:10271C0020202AF87F2B2028F322922480CF286EA9
:10272C00756C6C2900D22312240D3023F8C2237847
:10273C003D30D50108F60224B32D504349581224DC
:10274C000D2403B405004001E4902745931224396D
:0D275C00743A122439D225753D04022598E7
:10381D008B308A318932E4F53CF53BF53AF539F5D3
:10382D0037F538E534453545336012EBC0E0EAC075
:10383D00E0E9C0E0AB33AA34A935122CBBAB30059F
:10384D0032E532AA317002053114F9122A85F53D9F
:10385D00C394094007E53DD3940D40E1E53D642057
:10386D0060DBE53DB42D054338038016E53DB42BF3
:10387D0005433801800C74FF2532F53274FF353164
:10388D00F531E53660046410703FAB30AA31A932D2
:10389D00122A8564306009E536702E75360A802946
:1038AD00900001122A9EFF64786004EFB458134310
:1038BD00380175361074022532F532E43531F531A3
:1038CD008007E5367003753608AB300532E532AA50
:1038DD00317002053114F9122A85F53DC39461400A
:1038ED000AE53DD3947A5003533DDF74D0253DF561
:1038FD003DC3940A400CE53D9411406D74F9253D8E
:10390D00F53DE53DD395365060433801853C418505
:10391D003B40853A3F85393EAF367E00E4FCFDAB3A
:10392D003CAA3BA93AA839122C5CC8ECC8C9EDC910
:10393D00CAEECACBEFCBE4FCFDFEEB253DF53CEE2C
:10394D003AF53BED39F53AEC38F539AF3CAE3BADD8
:10395D003AFCAB41AA40A93FA83ED3122BFC500321
:10396D000238D64338040238D6E53820E003E48027
:10397D002DE53445354533601EAB30E53224FFF976
:10398D00E53134FFFAEBC0E0EAC0E0E9C0E0AB336B
:10399D00AA34A935122CBBE53830E20774FFFFFEBF
:1039AD00FDFC22E538AF3CAE3BAD3AAC3930E1031E
:0439BD00022BEE22C9
:102C4A00BB010689828A83F0225002F722BBFE0169
:022C5A00F32263
:102C5C00E88FF0A4CC8BF0A42CFCE98EF0A42CFC17
:102C6C008AF0EDA42CFCEA8EF0A4CDA8F08BF0A495
:102C7C002DCC3825F0FDE98FF0A42CCD35F0FCEBF4
:102C8C008EF0A4FEA9F0EB8FF0A4CFC5F02ECD39B9
:0F2C9C00FEE43CFCEAA42DCE35F0FDE43CFC2226
:102CAB00FAE6FB0808E6F925F0F618E6CA3AF6222A
:102CBB00BB011A89828A83D0F0D0E0F8D0E0F9D03A
:102CCB00E0FAD0E0FBE8C0E0C0F0022D395016E985
:102CDB00F8D083D082D0E0F9D0E0FAD0E0FBC0820C
:102CEB00C083022D30BBFE16E9F8D083D082D0E032
:0F2CFB00F9D0E0FAD0E0FBC082C083022D422264
:102D0A00D083D082F8E4937012740193700DA3A358
:102D1A0093F8740193F5828883E47374029368606C
:062D2A00EFA3A3A380DF6C
:092D3000EBF608EAF608E9F622C8
:092D3900EBF0A3EAF0A3E9F0229B
:092D4200EBF208EAF208E9F222C2
:00000001FF
